:1000000000308A00122C0000FF00030E8301A100C3
:100010007F08A0000A08A8008A01A00E0408A20018
:100020007708A3007808A4007908A5007A08A6003C
:100030007B08A700831383128C308400001D2228C4
:100040000C193528220884002308F7002408F8003A
:100050002508F9002608FA002708FB0028088A006E
:10006000210E8300FF0E7F0E09002F08183C031C91
:10007000C7281608AC001508AB002A082C02031C80
:100080005128031D47282B08290203185128290845
:100090002B02AD002C08AE002A08031C2A0FAE026A
:1000A0005E282A08FA00FA092908FF3A2B07AD0052
:1000B0002C08AE000318AE0A7A08AE072E08053CDD
:1000C0000318C728FF3A031D69282D08403C031870
:1000D000C7282C08AA002B08A9002E080A3C031CDC
:1000E0007E28031D77282D08EF3C031C7E2803146F
:1000F000B10DB20DB30DB40DAF0AC7282E08143CD4
:10010000031C9528031D88282D084F3C031C9528A7
:100110000310B10DB20DB30DB40D0314B10DB20D3A
:10012000B30DB40D0230AF07C7282E081D3C031CC9
:10013000B128031D9F282D08AF3C031CB1280310D4
:10014000B10DB20DB30DB40D0310B10DB20DB30D61
:10015000B40D0314B10DB20DB30DB40D0330AF07E0
:10016000C7280310B10DB20DB30DB40D0310B10DBE
:10017000B20DB30DB40D0310B10DB20DB30DB40D2E
:100180000314B10DB20DB30DB40D0430AF070C1153
:100190008A1122286E30840000080319DC280230FE
:1001A000F800F701F70BD228F80BD1289730F700A9
:1001B000F70BD828800BCF28003485170614ED01E3
:1001C0005E086D020318EB280A30F700F70BE628EB
:1001D0000000ED0AE02806108614ED015F086D02AC
:1001E0000318F9280A30F700F70BF4280000ED0A8D
:1001F000EE2886100615ED0160086D020318072928
:100200000A30F700F70B02290000ED0AFC2806115E
:100210000616ED0161086D02031815290A30F70072
:10022000F70B10290000ED0A0A2906120517ED0147
:1002300062086D02031823290A30F700F70B1E2904
:100240000000ED0A1829051385130830EE00CA20B6
:1002500000340030F8001F08C73978049F002130AF
:10026000F700F70B31291F151F1934291E08F70055
:100270000310F70C7708193EE7000310050CE8009F
:1002800008306802FA3E0318F729063E232A0317AE
:100290008E018D010313530803178C0083168C13F2
:1002A0000C15831203130B08F7008B138316031727
:1002B00055308D00AA308D008C148C185D290C11DE
:1002C0007708831203138B0403178E0101308D000E
:1002D0000313540803178C0083168C130C15831218
:1002E00003130B08F7008B138316031755308D008B
:1002F000AA308D008C148C187B290C11770883127E
:1003000003138B0403178E0102308D000313520870
:1003100003178C0083168C130C15831203130B0820
:10032000F7008B138316031755308D00AA308D000C
:100330008C148C1899290C117708831203138B04E1
:1003400003178E0103308D000313510803178C002F
:1003500083168C130C15831203130B08F7008B13F1
:100360008316031755308D00AA308D008C148C181D
:10037000B7290C117708831203138B0403178E011E
:1003800004308D0003135D0803178C0083168C1353
:100390000C15831203130B08F7008B138316031736
:1003A00055308D00AA308D008C148C18D5290C1175
:1003B0007708831203138B048601222A6708D3006F
:1003C00020308600F7296708D40040308600F729DE
:1003D0006708D20060308600F7296708D1008030B6
:1003E0008600F7296708DD00A0308600F72906306F
:1003F0005102D50006305107D60006305302D9000D
:1004000006305307DA0008305202D700083052078E
:10041000D80008305402DB0008305407DC005308D1
:10042000DE005408DF005208E0005108E1005D08DA
:10043000E200E7016708043C031C212ADD20E70AEB
:100440001A2A29290B2D0A108A140A118207472912
:10045000DE29E329E829ED29F229E801861D472A4A
:10046000E80A6808FA3C0318372AFA30E800031053
:10047000050CB000300EE900E90DE030E90569082F
:1004800086000A30F700F70B432A00002E2AE70106
:1004900086195B2AE70A0310050CB000300EE9004C
:1004A000E90DE030E905690886000A30F700F70B2E
:1004B000572A0000482A6708133C0318E801680817
:1004C000F93C03182D2A1608AA001508A900AF0147
:1004D00000340230E002DD206A08DF005F086B02B2
:1004E0000318762AE003DD20DF036E2A0034023091
:1004F000DF07DD206A08E0006B0860020318842A29
:10050000DF0ADD20E00A7C2A00345308DE005408AC
:10051000DF005108E1005408EA005B08EB006922A3
:10052000E9016908043C031C982ADD20E90A912AA4
:100530000230E0075108E100560861020318A42ABE
:10054000DD20DE0AE10A9C2AE80167086802031838
:10055000C92A5708EA005808EB0077225608E1003C
:10056000610855020318B82ADD20DE03E103B02A32
:100570005C08EA005B08EB0069225508E1005608B8
:1005800061020318C72ADD20DE0AE10ABF2AE80A51
:10059000A52A5708EA005208EB0077225608E10026
:1005A000510861020318D82ADD20DE03E103D02AB6
:1005B0005308DE005408DF005208E000E901690832
:1005C000043C031CE62ADD20E90ADF2A612E5308D9
:1005D000DE005408DF005208E0005408EA005B081F
:1005E000EB0069225108E100610855020318FC2A5A
:1005F000DD20DE03E103F42AE8016708680203183E
:10060000212B5708EA005808EB0077225508E10033
:10061000560861020318102BDD20DE0AE10A082BC0
:100620005C08EA005B08EB0069225608E1006108FB
:10063000550203181F2BDD20DE03E103172BE80A08
:10064000FD2A5708EA005208EB0077225508E1001E
:10065000510861020318302BDD20DE0AE10A282B45
:100660005408DF005308DE00E9016908043C031C5C
:100670003C2BDD20E90A352B652E5408DF00540899
:10068000EA005B08EB0069225108E10056086102AC
:1006900003184D2BDD20E10A462BE80167086802AC
:1006A0000318702B5708EA005808EB007722560809
:1006B000E100610855020318602BDD20E103592B8E
:1006C0005C08EA005B08EB0069225508E100560867
:1006D000610203186E2BDD20E10A672BE80A4E2B1E
:1006E0005108E1005708EA005208EB00772256084B
:1006F000E100610851020318802BDD20E103792B12
:100700005408DF00E9016908043C031C8A2BDD2042
:10071000E90A832B692E5408DF005208EA005808C2
:10072000EB0077225308DE005E08590203189B2B6A
:10073000DD20DE03942BE801670868020318BE2B56
:100740005C08EA005B08EB0069225908DE005A08E1
:100750005E020318AE2BDD20DE0AA72B5708EA0045
:100760005808EB0077225A08DE005E085902031889
:10077000BC2BDD20DE03B52BE80A9C2B5308DE00E2
:100780005C08EA005408EB006922E9016908043CAE
:10079000031CCD2BDD20E90AC62B6D2E5308DE008D
:1007A0005408DF005108E1005408EA005B08EB0040
:1007B0006922E9016908093C031CE12BDD20E90AF3
:1007C000DA2BE801670868020318022C5708EA00D0
:1007D0005808EB007722E9016908093C031CF32B58
:1007E000DD20E90AEC2B5C08EA005B08EB006922DB
:1007F000E9016908093C031C002CDD20E90AF92BFA
:10080000E80AE22B5708EA005208EB007722540866
:10081000DF00E9016908093C031C112CDD20E90A0D
:100820000A2C712E84011F308305063083169F0029
:1008300070308F008312A901AA01AB01AC01AD0198
:10084000AE01AF01B001B101B201B301B401B50114
:10085000B601B701B801B901BA01BB01BC01BD01C4
:10086000BE01BF01C001C101C201C301C401C50174
:10087000C601C701C801C901CA01CB01CC01CD0124
:10088000CE01CF01D001D101D201D301D401D501D4
:10089000D601D701D801D901DA01DB01DC01DD0184
:1008A000DE01DF01E001E101E2011F308316850076
:1008B000083086000E309F0083121F0838398138B7
:1008C0009F009701043097008530900083160C1527
:1008D000C03083128B04860103178E018D018316AD
:1008E0008C130C1483120C080313D300530F7A2CAF
:1008F0005030D30003178E0101308D0083168C1306
:100900000C1483120C080313D400540F892C50309C
:10091000D40003178E0102308D0083168C130C1443
:1009200083120C080313D200520F982C5030D200BF
:1009300003178E0103308D0083168C130C14831261
:100940000C080313D100510FA72C5030D10003170E
:100950008E0104308D0083168C130C1483120C0846
:100960000313DD005D0FB62C5030DD000630510260
:10097000D50006305107D60006305302D9000630A4
:100980005307DA0008305202D70008305207D80067
:1009900008305402DB0008305407DC005308DE0046
:1009A0005408DF005208E0005108E1005D08E20051
:1009B0000530E300E5016508063C031CFF2CE4015B
:1009C0006408033C031CFD2C650DF700F70DFC309B
:1009D000F70577086407353E840003178E0103137B
:1009E000630803178D0083168C130C1483120C08F4
:1009F00080000313E30AE40AE02CE50ADB2CE301A0
:100A00006308313C031C072DDD20E30A002D050897
:100A10000F3C031C29292D223008073C0318192EEE
:100A20002D22B00803195D2D3008073C031C5C2DF6
:100A30003008E500B003E4016408033C031C262DE4
:100A40003130640784008001E40A1C2D0314B10DC9
:100A5000B20DB30DB40D1E30EE00CA20E4016408DF
:100A6000033C031C472D300DF700F70DFC30F70554
:100A700077086407353EE8003130640784000008D9
:100A8000E9006808840069088000E40A2F2DE3016A
:100A90006308013C031C5C2D650EE700E70DE030A8
:100AA000E70567088600C830EE00CA208601C83016
:100AB000EE00CA20E30A482D102D2D223008073CF5
:100AC000031CB32DE3016308033C031C6D2D31307F
:100AD000630784008001E30A632D0314B10DB20D96
:100AE000B30DB40D1E30EE00CA20E501E401640828
:100AF000033C031C912D650DF700F70DFC30F70545
:100B000077086407353E84000008E8003130640748
:100B100084000008680203198F2DE50A912DE40A6C
:100B2000772D6408043C031DAE2DE3016308013CEE
:100B3000031CAD2D01306507F700770EE800E80DC6
:100B4000E030E80568088600C830EE00CA2086015B
:100B5000C830EE00CA20E30A962DB22D6508063C87
:100B60000318762D5D2D3008083C0319B82D102D83
:100B70000530E300E5016508063C031C052E013045
:100B80006507F700770EE800E80DE030E805680833
:100B90008600E4016408033C031CFC2D650DF7008E
:100BA000F70DFC30F70577086407353E8400000830
:100BB000E60003178E010313630803178D00031368
:100BC000660803178C0083168C130C15831203130D
:100BD0000B08F7008B138316031755308D00AA30CE
:100BE0008D008C148C18F22D0C11770883120313CE
:100BF0008B04E30AE40ACA2D0230E7009630EE00C7
:100C0000CA20E70BFE2DE50ABB2DE4016408013C78
:100C1000031C192EE03086000230E7009630EE000B
:100C2000CA20E70B0E2E86016430EE00CA20E40ACB
:100C3000062EE3016308313C031C242EDD20143012
:100C4000EE00CA20E30A1A2E2D22E3016308033CBA
:100C5000031C302E3130630784008001E30A262E06
:100C60000314B10DB20DB30DB40D1E30EE00CA2049
:100C7000E501E4016408033C031C542E650DF700F4
:100C8000F70DFC30F70577086407353E840000084F
:100C9000E800313064078400000868020319522E0E
:100CA000E50A542EE40A3A2E6408043C031DA32EE0
:100CB0006508F93E0318A22E073EA92E0230E70070
:100CC000852AA22E0230E700E72AA22E0230E70092
:100CD0003D2BA22E0230E7008B2BA22E0230E70024
:100CE000CE2BA22E5D086202031D812E5D08E2005C
:100CF00014305D0762020318802EDD20E20A782E90
:100D0000882E62085D020318882EE203DD20812E02
:100D1000A22E5D086202031D9A2E5D08E2001430C7
:100D20005D0262020319992E031C992EDD20E20355
:100D30008F2EA12E5D0862020318A12EE20ADD208B
:100D40009A2EA22EA72E6508063C0318392E242EB3
:100D500063000A108A140A1582075E2E622E662E20
:080D60006A2E6E2E722E892E00
:02400E00302F51
:00000001FF
